:020000040800F2
:1000000000060020A1020008AD0F00082D0F000817
:10001000850F00082D0F0008590F0008A3020008E3
:10002000A3020008A3020008A3020008FD220008A2
:10003000A3020008A3020008A3020008A30200080C
:10004000A3020008A3020008A3020008A3020008FC
:10005000A3020008A302000885370008B137000892
:10006000DD3700080938000835380008A302000809
:10007000A3020008A3020008A3020008A3020008CC
:10008000A3020008A3020008A3020008A3020008BC
:10009000A3020008A3020008A302000861380008B8
:1000A000A3020008A3020008A3020008A30200089C
:1000B000A3020008A3020008A3020008A30200088C
:1000C000A3020008A3020008A3020008A30200087C
:1000D000A3020008A3020008A3020008A30200086C
:1000E000C5380008A3020008A3020008A302000804
:1000F000A3020008A3020008A3020008A30200084C
:10010000A3020008A302000839390008A30200086E
:10011000A3020008A3020008A3020008A30200082B
:10012000A3020008A3020008A3020008A30200081B
:10013000A3020008A3020008A3020008A30200080B
:10014000A3020008A3020008A3020008A3020008FB
:10015000A3020008A3020008A3020008A3020008EB
:10016000A3020008A3020008A3020008A3020008DB
:10017000A3020008692E0008A3020008A3020008D9
:10018000A3020008A3020008A3020008A3020008BB
:10019000A3020008A3020008A3020008A3020008AB
:1001A000A3020008A3020008A3020008A30200089B
:1001B000A3020008A3020008A3020008A30200088B
:1001C000A3020008A3020008A3020008A30200087B
:1001D000A3020008552E0008A3020008A30200088D
:1001E000A3020008A3020008A3020008A30200085B
:1001F000A3020008A3020008A3020008A30200084B
:10020000A3020008A3020008A3020008A30200083A
:10021000A3020008A3020008A3020008A30200082A
:10022000A3020008A3020008A3020008A30200081A
:10023000A3020008A3020008A3020008A30200080A
:10024000A3020008A3020008A3020008A3020008FA
:10025000A3020008A3020008A3020008A3020008EA
:10026000A3020008A3020008A3020008A3020008DA
:10027000A3020008A3020008A3020008A3020008CA
:10028000A3020008A3020008A3020008A3020008BA
:10029000A3020008A3020008A3020008A3020008AA
:1002A00002E000F000F8FEE772B63A4880F30888F2
:1002B000394880F3098839484EF60851CEF20001DA
:1002C000086040F20000CCF200004EF63471CEF22D
:1002D00000010860BFF34F8FBFF36F8F40F2000043
:1002E000C0F2F0004EF68851CEF200010860BFF374
:1002F0004F8FBFF36F8F4FF00000E1EE100A4EF604
:100300003C71CEF200010860062080F31488BFF330
:100310006F8F02F0B1F802F053F802F0EDFF4FF0EA
:1003200055301F491B4A91423CBF41F8040BFAE784
:100330001C49194A91423CBF41F8040BFAE71A499B
:100340001A4A1B4B9A423EBF51F8040B42F8040B69
:10035000F8E700201749184A91423CBF41F8040BC6
:10036000FAE702F06BF803F04BF8144C144DAC4272
:1003700003DA54F8041B8847F9E700F041F8114C00
:10038000114DAC4203DA54F8041B8847F9E702F038
:1003900053B80000000600200022002000000008E2
:1003A0000000002000060020003D00080022002080
:1003B0005C220020602200207C420020A002000875
:1003C000A0020008A0020008A00200082DE9F04FDA
:1003D0002DED108AC1F80CD0D0F80CD0BDEC108AED
:1003E000BDE8F08F002383F311882846A047002042
:1003F00001F068FBFEE701F0E3FA00DFFEE7000032
:1004000038B500F0CDFC30B1164B00220E211A7227
:100410005A729972DA7201F031FF054601F064FFF9
:100420000446D0B9104B9D4219D001339D4241F290
:10043000883512BF044600250124002001F028FF62
:100440000CB100F059F800F045FD00F0E3FB284640
:1004500000F004F900F050F8F9E70025EDE7054653
:10046000EBE700BF00220020010007B008B500F054
:10047000A3FBA0F120035842584108BD07B541F243
:100480001203022101A8ADF8043000F0B3FB03B061
:100490005DF804FB202310B583F311881248C3686C
:1004A0000BB101F095FB0023104A4FF47A710E480E
:1004B00001F052FB002383F311880D4C236813B124
:1004C0002368013B2360636813B16368013B636089
:1004D000084B1B7833B9636823B9022000F074FC21
:1004E0003223636010BD00BF602200209504000825
:1004F0007C23002074220020F8B5514B514A1C4641
:100500001968013100F09B8004339342F8D162688E
:100510004D4B9A4240F293804C4B9B6803F1006331
:1005200003F500339A4280F08A80002000F098FBA7
:100530000220474B187000F03DFC464B0021D3F8D9
:10054000E820C3F8E810D3F81021C3F81011D3F84D
:100550001021D3F8EC20C3F8EC10D3F81421C3F821
:100560001411D3F81421D3F8F020C3F8F010D3F805
:100570001821C3F81811D3F81821D3F8802042F0BD
:100580000062C3F88020D3F8802022F00062C3F814
:100590008020D3F88020D3F8802042F00072C3F886
:1005A0008020D3F8802022F00072C3F88020D3F896
:1005B000803072B64FF0E023C3F8084DD4E9000450
:1005C000BFF34F8FBFF36F8F234AC2F88410BFF37E
:1005D0004F8F536923F480335361BFF34F8FD2F8A9
:1005E000803043F6E076C3F3C905C3F34E335B01B5
:1005F00003EA060C29464CEA81770139C2F8747285
:10060000F9D2203B13F1200FF2D1BFF34F8FBFF38C
:100610006F8FBFF34F8FBFF36F8F536923F4003396
:1006200053610023C2F85032BFF34F8FBFF36F8F77
:10063000202383F31188854680F308882047F8BD7E
:100640000000020820000208FFFF0108002200202D
:10065000742200200044025800ED00E02DE9F04F24
:1006600093B0A94B2022FF2100900AA89D6800F0BA
:10067000DBFBA64A1378A3B90121A5481170C3601A
:10068000202383F31188C3680BB101F0A1FA002382
:10069000A04A4FF47A719E4801F05EFA002383F37A
:1006A0001188009B9C4A03B1136000239B49009C66
:1006B00098469B461E469A460B705360012000F0F8
:1006C00079FB24B1944B1B68002B00F016820020AC
:1006D00000F072FA0390039B002BF2DB012000F084
:1006E00061FB039B213B162BE8D801A252F823F0B3
:1006F0004D0700087507000809080008BD06000836
:10070000BD060008BD0600089D0800086F0A000825
:1007100089090008EB090008130A0008390A0008D3
:10072000BD0600084B0A0008BD060008BD0A000807
:10073000ED070008BD060008010B00085907000876
:10074000ED070008BD060008EB0900080220FFF7CE
:100750008DFE002840F0FB81009B022105A8B8F126
:10076000000F08BF1C4641F21233ADF8143000F000
:1007700041FAA3E74FF47A7000F01EFA071EEBDB94
:100780000220FFF773FE0028E6D0013F052F00F29C
:10079000E081DFE807F0030A0D101336052304217A
:1007A00005A8059300F026FA17E004215648F9E75A
:1007B00004215B48F6E704215A48F3E74FF01C098F
:1007C000484609F1040900F04DFA0421059005A8F6
:1007D00000F010FAB9F12C0FF2D101204FF0000A0D
:1007E00000FA07F747EA0B0B5FFA8BFB00F068FB98
:1007F00026B10BF00B030B2B08BF0024FFF73EFEC6
:100800005CE704214848CDE7002EA5D00BF00B0390
:100810000B2BA1D10220FFF729FE074600289BD011
:1008200001203E4E00F01CFA4FF00008022030700C
:1008300000F0C0FA5FFA88F9484600F021FA044651
:1008400090B1484608F1010800F02AFA0028F1D1D9
:10085000B846044641F21213022105A83E46ADF8FF
:10086000143000F0C7F929E7012325460220337030
:1008700000F098FA244B9B68AB4207D9284600F059
:10088000F1F9013040F068810435F3E70025234B8E
:10089000B8463E461D70204B5D60A7E7002E3FF432
:1008A0005BAF0BF00B030B2B7FF456AF02201B4BFF
:1008B000187000F07FFA322000F07EF9B0F10009E4
:1008C000FFF64AAF19F003077FF446AF0E4A09EB73
:1008D0000503926893423FF63FAFB9F5807F3FF73B
:1008E0003BAF124BB945019322DD4FF47A7000F013
:1008F00063F90390039A002AFFF62EAF039A01379B
:10090000019B03F8012BEDE7002200207823002053
:1009100060220020950400087C230020742200201F
:1009200004220020082200200C220020782200202F
:10093000C820FFF79BFD074600283FF40DAF1F2D91
:1009400011D8C5F120020AAB25F0030084494A45BD
:10095000184428BF4A46019200F040FA019AFF214C
:100960007F4800F061FA4FEAA903C9F387027C4986
:100970002846019300F060FA064600283FF46AAF6B
:10098000019B05EB830531E70220FFF76FFD00288F
:100990003FF4E2AE00F0A0F900283FF4DDAE0027FE
:1009A000B946704B9B68BB4218D91F2F11D80A9BC0
:1009B00001330ED027F0030312AA134453F8203C4E
:1009C00005934846042205A9043700F0F1FA814650
:1009D000E7E7384600F046F90590F2E7CDF81490C5
:1009E000042105A800F006F900E70023642104A80B
:1009F000049300F0F5F800287FF4AEAE0220FFF774
:100A000035FD00283FF4A8AE049800F05BF905908E
:100A1000E6E70023642104A8049300F0E1F800282D
:100A20007FF49AAE0220FFF721FD00283FF494AE38
:100A3000049800F049F9EAE70220FFF717FD0028C3
:100A40003FF48AAE00F058F9E1E70220FFF70EFD0F
:100A500000283FF481AE05A9142000F053F90746A1
:100A60000421049004A800F0C5F83946B9E7322003
:100A700000F0A2F8071EFFF66FAEBB077FF46CAE66
:100A8000384A07EB0A03926893423FF665AE0220AC
:100A9000FFF7ECFC00283FF45FAE27F00307574454
:100AA000BA453FF4A3AE50460AF1040A00F0DAF862
:100AB0000421059005A800F09DF8F1E74FF47A7045
:100AC000FFF7D4FC00283FF447AE00F005F90028FA
:100AD00044D00A9B01330BD008220AA9002000F061
:100AE000ABF900283AD02022FF210AA800F09CF997
:100AF000FFF7C4FC1C4800F0EBFF13B0BDE8F08F1B
:100B0000002E3FF429AE0BF00B030B2B7FF424AE29
:100B10000023642105A8059300F062F80746002829
:100B20007FF41AAE0220FFF7A1FC814600283FF4B3
:100B300013AEFFF7A3FC41F2883000F0C9FF05981F
:100B400000F0F2F94E463C4600F0BAF9B6E506462A
:100B50004CE64FF0000AFFE5B8467BE6374679E6FB
:100B60007822002000220020A08601000F4B70B5E3
:100B70001B780C460133DBB2012B11D80C4D4FF41E
:100B80007A732968A2FB033222460E6A0146284680
:100B9000B047844204D1074B002201201A7070BD77
:100BA0004FF4FA7000F094FF0020F8E710220020C4
:100BB00070250020B0230020002307B50246012144
:100BC0000DF107008DF80730FFF7D0FF20B19DF839
:100BD000070003B05DF804FB4FF0FF30F9E70000B9
:100BE0000A46042108B5FFF7C1FF80F00100C0B23A
:100BF000404208BD30B4054C0A46014623682046F1
:100C0000DD69034BAC4630BC604700BF7025002057
:100C1000A086010070B5104C0025104E01F006FAB8
:100C200020803068238883420CD800252088013832
:100C300001F0F8F923880544013BB5F5802F2380A6
:100C4000F4D370BD01F0EEF9336805440133B5F516
:100C5000003F3360E5D3E8E7B2230020842300207F
:100C600001F0C2BA00F1006000F500300068704782
:100C700000F10060920000F5003001F039BA000088
:100C8000054B1A68054B1B889B1A834202D91044F6
:100C900001F0C8B90020704784230020B22300204F
:100CA00038B5074D04462868204401F0C1F928B939
:100CB00028682044BDE8384001F0CCB938BD00BFF9
:100CC000842300200020704700F1FF5000F58F10B2
:100CD000D0F8000870470000064991F8243033B17D
:100CE00000230822086A81F82430FFF7C1BF0120E1
:100CF000704700BF88230020014B1868704700BF71
:100D00000010005C244BF0B51A680446234BC2F374
:100D10000B06120C1F885868BE4293F9085028D061
:100D20009F89BE4206D101200C2505FB003358687F
:100D300093F9085041F201039A421CD041F2030397
:100D40009A421AD042F201039A4218D042F20303A7
:100D50009A4208BF5625621E0B46441E0A4493421F
:100D60000FD214F9016F581C6EB1034600F8016CE4
:100D7000F5E70020D8E75A25EDE75925EBE7582598
:100D8000E9E7184605E02C2482421C7001D9981C22
:100D90005D70401AF0BD00BF0010005C14220020FE
:100DA00000207047022802D1014B04229A6170474B
:100DB00000080258022803D1024B4FF480229A61A6
:100DC000704700BF00080258022804D1024A536944
:100DD00083F004035361704700080258002310B5E4
:100DE000934203D0CC5CC4540133F9E710BD00003A
:100DF000013810B510F9013F3BB191F900409C4218
:100E000003D11AB10131013AF4E71AB191F9002086
:100E1000981A10BD1046FCE703460246D01A12F994
:100E2000011B0029FAD1704702440346934202D0C5
:100E300003F8011BFAE770472DE9F8431F4D1446EC
:100E40000746884695F8242052BBDFF870909CB383
:100E500095F824302BB92022FF2148462F62FFF756
:100E6000E3FF95F824004146C0F1080205EB80003D
:100E7000A24228BF2246D6B29200FFF7AFFF95F8F4
:100E80002430A41B17441E449044E4B2F6B2082E4A
:100E900085F82460DBD1FFF71FFF0028D7D108E0D9
:100EA0002B6A03EB82038342CFD0FFF715FF0028A4
:100EB000CBD10020BDE8F8830120FBE78823002088
:100EC000024B1A78024B1A70704700BFB023002003
:100ED0001022002010B5104C104800F0FBF82146FD
:100EE0000E4800F023F924680D48D4F89020D2F879
:100EF000043843F00203C2F8043800F0E9FD094960
:100F0000204600F021FAD4F89020D2F8043823F0DB
:100F10000203C2F8043810BDE43A0008702500202E
:100F200040420F00EC3A00087047000000B59BB04B
:100F3000EFF3098168226846FFF750FFEFF305835E
:100F4000044B9A6BDA6A9A6A9A6A9A6A9A6A9A6AF5
:100F50009B6AFEE700ED00E000B59BB0EFF309816E
:100F600068226846FFF73AFFEFF30583044B9A6B5C
:100F70009A6A9A6A9A6A9A6A9A6A9B6AFEE700BFB4
:100F800000ED00E000B59BB0EFF3098168226846F0
:100F9000FFF724FFEFF30583034B5A6B9A6A9A6AB3
:100FA0009A6A9A6A9B6AFEE700ED00E0FEE700009D
:100FB00030B50A44084D91420DD011F8013B58401C
:100FC000082340F30004013B2C4013F0FF0384EAA4
:100FD0005000F6D1EFE730BD2083B8ED02684368DA
:100FE0001143016003B118477047000013B5406B0F
:100FF00000F58054D4F8A4381A681178042914D163
:10100000017C022911D11979012312898B401342E5
:101010000BD101A94C3002F06FF8D4F8A448024675
:10102000019B2179206800F0DFF902B010BD0000BB
:10103000143001F0F1BF00004FF0FF33143001F025
:10104000EBBF00004C3002F0C3B800004FF0FF339C
:101050004C3002F0BDB80000143001F0BFBF0000FA
:101060004FF0FF31143001F0B9BF00004C3002F0F6
:101070008FB800004FF0FF324C3002F089B800000A
:101080000020704710B500F58054D4F8A4381A68D1
:101090001178042917D1017C022914D1597901232F
:1010A00052898B4013420ED1143001F051FF024699
:1010B00048B1D4F8A4484FF4407361792068BDE882
:1010C000104000F07FB910BD406BFFF7DBBF0000A0
:1010D000704700007FB5124B0125042604460360CB
:1010E0000023057400F1840243602946C0E90233FD
:1010F0000C4B0290143001934FF44073009601F0B2
:1011000003FF094B04F69442294604F14C00029473
:10111000CDE900634FF4407301F0CAFF04B070BD25
:10112000203A0008C9100008ED0F00080A682023C3
:1011300083F311880B790B3342F823004B79133377
:1011400042F823008B7913B10B3342F8230000F5EA
:101150008053C3F8A41802230374002383F3118877
:101160007047000038B5037F044613B190F854303F
:10117000ABB90125201D0221FFF730FF04F1140057
:101180006FF00101257700F0CBFC04F14C0084F8EE
:1011900054506FF00101BDE8384000F0C1BC38BDCB
:1011A00010B5012104460430FFF718FF0023237710
:1011B00084F8543010BD000038B5044600251430C2
:1011C00001F0BAFE04F14C00257701F089FF201DE3
:1011D00084F854500121FFF701FF2046BDE8384054
:1011E000FFF750BF90F8803003F06003202B06D14A
:1011F00090F881200023212A03D81F2A06D8002036
:101200007047222AFBD1C0E91D3303E0034A42673D
:1012100007228267C3670120704700BF2C2200208D
:1012200037B500F58055D5F8A4381A681178042927
:101230001AD1017C022917D11979012312898B4017
:10124000134211D100F14C04204602F009F858B1C4
:1012500001A9204601F050FFD5F8A4480246019BA1
:101260002179206800F0C0F803B030BD01F10B0314
:10127000F0B550F8236085B004460D46FEB120233A
:1012800083F3118804EB8507301D0821FFF7A6FEC4
:10129000FB6806F14C005B691B681BB1019001F013
:1012A00039FF019803A901F027FF024648B1039BCB
:1012B0002946204600F098F8002383F3118805B0F2
:1012C000F0BDFB685A691268002AF5D01B8A013B01
:1012D0001340F1D104F18002EAE70000133138B580
:1012E00050F82140ECB1202383F3118804F580539A
:1012F000D3F8A4281368527903EB8203DB689B6957
:101300005D6845B104216018FFF768FE294604F1C5
:10131000140001F027FE2046FFF7B4FE002383F3FC
:10132000118838BD7047000001F01AB9012340222E
:10133000002110B5044600F8303BFFF775FD00238F
:10134000C4E9013310BD000010B52023044683F327
:1013500011882422416000210C30FFF765FD2046F2
:1013600001F020F902232370002383F3118810BDBC
:1013700070B500EB8103054650690E461446DA60ED
:1013800018B110220021FFF74FFDA06918B11022FB
:101390000021FFF749FD31462846BDE8704001F0C5
:1013A00013BA000083682022002103F0011310B556
:1013B000044683601030FFF737FD2046BDE810403B
:1013C00001F08EBAF0B4012500EB810447898D400D
:1013D000E4683D43A469458123600023A260636003
:1013E000F0BC01F0ABBA0000F0B4012500EB8104C1
:1013F00007898D40E4683D436469058123600023CB
:10140000A2606360F0BC01F021BB000070B5022354
:1014100000250446242203702946C0F888500C3069
:1014200040F8045CFFF700FD204684F8705001F09E
:101430005FF963681B6823B129462046BDE8704008
:10144000184770BD037880F88C300523037043681B
:101450001B6810B504460BB1042198470023A36014
:1014600010BD000090F88C20436802701B680BB11F
:10147000052118477047000070B590F87030044699
:1014800013B1002380F8703004F18002204601F08F
:101490004BFA63689B68B3B994F8803013F0600529
:1014A00035D00021204601F0F5FC0021204601F056
:1014B000E5FC63681B6813B10621204698470623A4
:1014C00084F8703070BD204698470028E4D0B4F806
:1014D0008630A26F9A4288BFA36794F98030A56FC7
:1014E000002B4FF0200380F20381002D00F0F280EA
:1014F000092284F8702083F3118800212046D4E962
:101500001D23FFF771FF002383F31188DAE794F8B6
:10151000812003F07F0343EA022340F20232934228
:1015200000F0C58021D8B3F5807F48D00DD8012BBD
:101530003FD0022B00F09380002BB2D104F188023F
:1015400062670222A267E367C1E7B3F5817F00F01B
:101550009B80B3F5407FA4D194F88230012BA0D1B9
:10156000B4F8883043F0020332E0B3F5006F4DD099
:1015700017D8B3F5A06F31D0A3F5C063012B90D875
:101580006368204694F882205E6894F88310B4F86B
:101590008430B047002884D0436863670368A3673A
:1015A0001AE0B3F5106F36D040F6024293427FF452
:1015B00078AF5C4B63670223A3670023C3E794F80B
:1015C0008230012B7FF46DAFB4F8883023F0020332
:1015D000A4F88830C4E91D55E56778E7B4F8803091
:1015E000B3F5A06F0ED194F88230204684F88A308B
:1015F00001F0DCF863681B6813B1012120469847AD
:10160000032323700023C4E91D339CE704F18B03FB
:1016100063670123C3E72378042B10D1202383F3CE
:1016200011882046FFF7BEFE85F311880321636809
:1016300084F88B5021701B680BB12046984794F8B2
:101640008230002BDED084F88B3004232370636853
:101650001B68002BD6D0022120469847D2E794F889
:10166000843020461D0603F00F010AD501F04EF923
:10167000012804D002287FF414AF2B4B9AE72B4BA0
:1016800098E701F035F9F3E794F88230002B7FF406
:1016900008AF94F8843013F00F01B3D01A06204637
:1016A00002D501F00FFCADE701F000FCAAE794F8C9
:1016B0008230002B7FF4F5AE94F8843013F00F01E4
:1016C000A0D01B06204602D501F0E4FB9AE701F00A
:1016D000D5FB97E7142284F8702083F311882B46FA
:1016E0002A4629462046FFF76DFE85F31188E9E674
:1016F0005DB1152284F8702083F311880021204603
:10170000D4E91D23FFF75EFEFDE60B2284F870206E
:1017100083F311882B462A4629462046FFF764FEAC
:10172000E3E700BF503A0008483A00084C3A000886
:1017300038B590F870300446002B3ED0063BDAB244
:101740000F2A34D80F2B32D8DFE803F037313108B5
:10175000223231313131313131313737856FB0F8A3
:1017600086309D4214D2C3681B8AB5FBF3F203FB9B
:1017700012556DB9202383F311882B462A4629463A
:10178000FFF732FE85F311880A2384F870300EE0EB
:10179000142384F87030202383F31188002320461B
:1017A0001A461946FFF70EFE002383F3118838BD51
:1017B000C36F03B198470023E7E70021204601F0FB
:1017C00069FB0021204601F059FB63681B6813B1D7
:1017D0000621204698470623D7E7000010B590F869
:1017E00070300446142B29D017D8062B05D001D809
:1017F0001BB110BD093B022BFBD80021204601F094
:1018000049FB0021204601F039FB63681B6813B1D6
:10181000062120469847062319E0152BE9D10B2312
:1018200080F87030202383F3118800231A4619466C
:10183000FFF7DAFD002383F31188DAE7C3689B69B9
:101840005B68002BD5D1C36F03B19847002384F8A0
:101850007030CEE7024B0022C3E900339A60704734
:10186000B4230020002382680374054B1B68996829
:101870009142FBD25A680360426010605860704722
:10188000B423002008B5202383F31188037C032BA5
:1018900005D0042B0DD02BB983F3118808BD436903
:1018A00000221A604FF0FF334361FFF7DBFF002394
:1018B000F2E7D0E9003213605A60F3E70023826850
:1018C0000374054B1B6899689142FBD85A68036002
:1018D0004260106058607047B4230020054B1969BE
:1018E00008741868026853601A6018610123037451
:1018F000FEF76CBDB42300204B1C30B5044687B006
:101900000A4D10D02B6901A8094A00F025F920469C
:10191000FFF7E4FF049B13B101A800F059F92B690C
:10192000586907B030BDFFF7D9FFF8E7B4230020AE
:101930008518000838B50C4D044641612B69816853
:101940009A68914203D8BDE83840FFF78BBF18462C
:10195000FFF7B4FF01232C61014623742046BDE844
:101960003840FEF733BD00BFB4230020044B1A6893
:101970001B6990689B68984294BF002001207047C3
:10198000B423002010B5084C236820691A685460FD
:101990002260012223611A74FFF790FF014620693B
:1019A000BDE81040FEF712BDB423002008B5FFF7D4
:1019B000DDFF18B1BDE80840FFF7E4BF08BD000037
:1019C000FFF7E0BFFEE7000010B50C4CFFF742FF49
:1019D00000F0B4F880220A49204600F03BF80123C9
:1019E00044F8180C037400F099FC002383F3118869
:1019F00062B60448BDE8104000F04CB8DC2300207B
:101A0000543A0008643A000800F01CB9EFF3118062
:101A100020B9EFF30583202282F31188704700007C
:101A200010B530B9EFF30584C4F3080414B180F3A2
:101A3000118810BDFFF7BAFF84F31188F9E70000A1
:101A4000034A516853685B1A9842FBD8704700BF3D
:101A5000001000E082600222028270478368A3F1D6
:101A60007C0243F80C2C026943F83C2C426943F891
:101A7000382C074A43F81C2CC268A3F1180043F81D
:101A8000102C022203F8082C002203F8072C7047C0
:101A9000E503000810B5202383F31188FFF7DEFF6C
:101AA00000210446FFF746FF002383F311882046F8
:101AB00010BD0000024B1B6958610F20FFF70EBFDD
:101AC000B4230020202383F31188FFF7F3BF000025
:101AD00008B50146202383F311880820FFF70CFF87
:101AE000002383F3118808BD49B1064B42681B6986
:101AF00018605A60136043600420FFF7FDBE4FF08A
:101B0000FF307047B42300200368984206D01A685B
:101B10000260506018465961FFF7A4BE704700008C
:101B200038B504460D462068844200D138BD0368AC
:101B300023605C604561FFF795FEF4E7054B4FF0CD
:101B4000FF3103F11402C3E905220022C3E90712A1
:101B5000704700BFB423002070B51C4E05460C46EC
:101B6000C0E9032301F0B2FB334653F8142F9A4225
:101B70000DD130620A2C2CBF00190A302A60C5E949
:101B80000124C6E90555BDE8704001F089BB316A02
:101B9000431AE31838BF1C469368A34202D90819B8
:101BA00001F08EFB73699A6894420CD85A68AC6055
:101BB0002B606A6015609A685D60121B9A604FF036
:101BC000FF33F36170BDA41A1B68ECE7B423002057
:101BD00038B51B4C636998420DD08168D0E900325A
:101BE00013605A600022C2609A680A449A604FF0FB
:101BF000FF33E36138BD03682246002142F8143FF9
:101C000093425A60C16003D1BDE8384001F052BB35
:101C10009A688168256A0A449A6001F057FB6369F3
:101C2000411B9A688A42E5D9AB181D1A206A092D12
:101C300098BF01F10A02BDE83840104401F040BBF2
:101C4000B42300202DE9F041184C002704F11406BC
:101C5000656901F03BFB236AAA68C11A8A4215D85C
:101C60001344D5F80C802362D5E9003213605A6022
:101C70006369EF60B34201D101F01CFB87F3118867
:101C80002869C047202383F31188E1E76169B142E5
:101C900009D013441B1ABDE8F0410A2B2CBFC01811
:101CA0000A3001F00DBBBDE8F08100BFB423002075
:101CB00000207047FEE70000704700004FF0FF3043
:101CC0007047000002290CD0032904D001290748DD
:101CD00018BF00207047032A05D8054800EBC20052
:101CE0007047044870470020704700BF483B000819
:101CF0003C220020FC3A000870B59AB00546084620
:101D0000144601A900F0C2F801A8FFF785F8431CAA
:101D10000022C6B25B001046C5E9003423700323DD
:101D2000023404F8013C01ABD1B202348E4201D836
:101D30001AB070BD13F8011B013204F8010C04F84D
:101D4000021CF1E708B5202383F311880348FFF74D
:101D500067FA002383F3118808BD00BF70250020B7
:101D600090F8803003F01F02012A07D190F88120FB
:101D70000B2A03D10023C0E91D3315E003F06003F3
:101D8000202B08D1B0F884302BB990F88120212A7B
:101D900003D81F2A04D8FFF725BA222AEBD0FAE786
:101DA000034A426707228267C3670120704700BF6A
:101DB0003322002007B5052917D8DFE801F01916EE
:101DC00003191920202383F31188104A012101905F
:101DD000FFF7CEFA019802210D4AFFF7C9FA0D4824
:101DE000FFF7EAF9002383F3118803B05DF804FBE1
:101DF000202383F311880748FFF7B4F9F2E7202383
:101E000083F311880348FFF7CBF9EBE79C3A00080E
:101E1000C03A00087025002038B50C4D0C4C2A46FD
:101E20000C4904F10800FFF767FF05F1CA0204F14D
:101E300010000949FFF760FF05F5CA7204F11800A8
:101E40000649BDE83840FFF757BF00BF483E0020B5
:101E50003C2200207C3A0008863A0008913A0008AB
:101E600070B5044608460D46FEF7D6FFC6B22046BA
:101E7000013403780BB9184670BD32462946FEF787
:101E8000B7FF0028F3D10120F6E700002DE9F84F55
:101E900005460C46FEF7C0FF2C49C6B22846FFF7A0
:101EA000DFFF08B10536F6B229492846FFF7D8FF0B
:101EB00008B11036F6B2632E0DD8DFF89080DFF847
:101EC0009090244FDFF894A0DFF894B02E7846B9B4
:101ED0002670BDE8F88F29462046BDE8F84F01F08E
:101EE00089BD252E2ED1072241462846FEF780FFC8
:101EF00070B9DBF8003007350C3444F80C3CDBF8E3
:101F0000043044F8083CDBF8083044F8043CDDE7D2
:101F1000082249462846FEF76BFF98B9A21C0E4BD3
:101F2000197802320909C95D02F8041C13F8011B73
:101F300001F00F015345C95D02F8031CF0D11834BC
:101F40000835C3E7013504F8016BBFE7683B0008BB
:101F5000913A00087D3B000800E8F11F0CE8F11FF2
:101F6000703B0008BFF34F8F044B1A695107FCD137
:101F7000D3F810215207F8D1704700BF002000525B
:101F800008B50D4B1B78ABB9FFF7ECFF0B4BDA68CC
:101F9000D10704D50A4A5A6002F188325A60D3F850
:101FA0000C21D20706D5064AC3F8042102F1883273
:101FB000C3F8042108BD00BFA64000200020005245
:101FC0002301674508B5114B1B78F3B9104B1A690B
:101FD000510703D5DA6842F04002DA60D3F81021E5
:101FE000520705D5D3F80C2142F04002C3F80C216A
:101FF000FFF7B8FF064BDA6842F00102DA60D3F867
:102000000C2142F00102C3F80C2108BDA6400020BB
:10201000002000520F289ABF00F580604004002085
:10202000704700004FF400307047000010207047E8
:102030000F2808B50BD8FFF7EDFF00F50033026855
:10204000013204D104308342F9D1012008BD0020BF
:10205000FCE700000F2870B5054645D8FFF7D6FC11
:10206000224CFFF77FFF0646FFF78AFF4FF0FF3352
:10207000072D6361C4F8143120D82361FFF772FF84
:102080002B0243F02403E360E36843F08003E36042
:1020900023695A07FCD42846FFF764FF4FF4003148
:1020A000FFF7B8FF00F002F93046FFF78BFFFFF7AC
:1020B000B7FC2846BDE87040FFF7BABFC4F810313E
:1020C000FFF750FFA5F108031B0243F02403C4F8F7
:1020D0000C31D4F80C3143F08003C4F80C31D4F83F
:1020E00010315B07FBD4D6E7002070BD0020005202
:1020F0002DE9F84F40EA020305460C461746D8067C
:1021000002D00020BDE8F88F27F01F07DFF8D4B019
:10211000FFF736FF2744BC4203D10120FFF752FFEF
:10212000F0E720222946204601F054FC10B9203562
:102130002034F0E72B4605F120021E68711CE0D127
:1021400004339A42F9D1FFF761FC05F17843234A41
:10215000B3F5801F224B28BF9A4603F1040338BF12
:102160009046A2F1080228BF9846A3F108033ABF9F
:102170009146DA469946FFF7F5FEC8F80060A5EBF0
:10218000040CD9F8002004F11C0142F00202C9F845
:102190000020221FDAF8006016F00506FAD152F886
:1021A000043F8A424CF80230F4D1BFF34F8FFFF75F
:1021B000D9FE4FF0FF32C8F80020D9F8002022F0F5
:1021C0000202C9F80020FFF72BFC202221462846F6
:1021D00001F000FC0028AAD030469FE714200052EE
:1021E000102100521020005210B5084C237828B15D
:1021F0001BB9FFF7C5FE0123237010BD002BFCD0D7
:102200002070BDE81040FFF7DDBE00BFA6400020F3
:102210000244074BD2B210B5904200D110BD441C0D
:1022200000B253F8200041F8040BE0B2F4E700BF1D
:10223000504000580E4B30B51C6F240405D41C6F61
:102240001C671C6F44F400441C670A4C024423685A
:10225000D2B243F480732360074B904200D130BD6B
:10226000441C51F8045B00B243F82050E0B2F4E79C
:1022700000440258004802585040005807B5012257
:1022800001A90020FFF7C4FF019803B05DF804FB2B
:1022900013B50446FFF7F2FFA04205D0012201A9C1
:1022A00000200194FFF7C6FF02B010BD0144BFF348
:1022B0004F8F064B884204D3BFF34F8FBFF36F8F0E
:1022C0007047C3F85C022030F4E700BF00ED00E087
:1022D000034B1A681AB9034AD2F8D0241A6070471F
:1022E000A84000200040025808B5FFF7F1FF024B5C
:1022F0001868C0F3806008BDA8400020EFF3098390
:10230000054968334A6B22F001024A6383F3098866
:10231000002383F31188704700EF00E0202080F352
:10232000118862B60D4B0E4AD96821F4E0610904A8
:10233000090C0A430B49DA60D3F8FC2042F08072A2
:10234000C3F8FC20084AC2F8B01F116841F001012F
:1023500011601022DA7783F82200704700ED00E068
:102360000003FA0555CEACC5001000E0202310B5DF
:1023700083F311880E4B5B6813F4006314D0F1EE05
:10238000103AEFF309844FF08073683CE361094B26
:10239000DB6B236684F30988FFF7E8FA10B1064B7C
:1023A000A36110BD054BFBE783F31188F9E700BF7C
:1023B00000ED00E000EF00E0F7030008FA0300087A
:1023C00070B5BFF34F8FBFF36F8F1A4A0021C2F869
:1023D0005012BFF34F8FBFF36F8F536943F4003335
:1023E0005361BFF34F8FBFF36F8FC2F88410BFF3F9
:1023F0004F8FD2F8803043F6E074C3F3C900C3F3C3
:102400004E335B0103EA0406014646EA8175013951
:10241000C2F86052F9D2203B13F1200FF2D1BFF382
:102420004F8F536943F480335361BFF34F8FBFF332
:102430006F8F70BD00ED00E0FEE700000A4B0B4817
:102440000B4A90420BD30B4BC11EDA1C121A22F01E
:1024500003028B4238BF00220021FEF7E5BC53F88F
:10246000041B40F8041BECE75C3D00087C420020A4
:102470007C4200207C4200207047000070B5D0E90B
:10248000244300224FF0FF359E6804EB42135101B4
:10249000D3F80009002805DAD3F8000940F080409D
:1024A000C3F80009D3F8000B002805DAD3F8000BB5
:1024B00040F08040C3F8000B013263189642C3F825
:1024C0000859C3F8085BE0D24FF00113C4F81C3878
:1024D00070BD000000EB8103D3F80CC02DE9F04380
:1024E000DCF814204E1CD0F89050D2F800E005EB38
:1024F000063605EB4118506870450AD30122D5F81D
:10250000343802FA01F123EA0101C5F83418BDE8B4
:10251000F083AEEB0003BCF81040A34228BF234673
:10252000D8F81849A4B2B3EB840FF0D89468A4F19A
:10253000040959F8047F3760A4EB09071F44042FEE
:10254000F7D81C44034494605360D4E7890141F0F8
:102550002001016103699B06FCD41220FFF770BAC9
:1025600010B50A4C2046FEF7E1FE094BC4F8903046
:10257000084BC4F89430084C2046FEF7D7FE074BB2
:10258000C4F89030064BC4F8943010BDAC40002025
:1025900000000840B43B000848410020000004400F
:1025A000C03B000870B503780546012B5DD1494B4F
:1025B000D0F89040984259D1474B0E216520D3F86E
:1025C000D82042F00062C3F8D820D3F8002142F0AE
:1025D0000062C3F80021D3F80021D3F8802042F034
:1025E0000062C3F88020D3F8802022F00062C3F894
:1025F0008020D3F8803000F071FC384BE360384B1A
:10260000C4F800380023D5F89060C4F8003EC02319
:1026100023604FF40413A3633369002BFCDA012316
:102620000C203361FFF70CFA3369DB07FCD412206E
:10263000FFF706FA3369002BFCDA00262846A6606D
:10264000FFF71CFF6B68C4F81068DB68C4F81468F7
:10265000C4F81C68002B3AD1224BA3614FF0FF3322
:102660006361A36843F00103A36070BD1E4B9842F1
:10267000C8D1194B0E214D20D3F8D82042F000725A
:10268000C3F8D820D3F8002142F00072C3F800212B
:10269000D3F80021D3F8802042F00072C3F88020E4
:1026A000D3F8802022F00072C3F88020D3F8802075
:1026B000D3F8D82022F08062C3F8D820D3F80021C4
:1026C00022F08062C3F80021D3F8003193E7074B72
:1026D000C3E700BFAC400020004402584014004053
:1026E00003002002003C30C048410020083C30C0BC
:1026F000F8B5D0F89040054600214FF0006620461E
:10270000FFF724FFD5F8941000234FF001128F68D3
:102710004FF0FF30C4F83438C4F81C2804EB4312DF
:1027200001339F42C2F80069C2F8006BC2F8080981
:10273000C2F8080BF2D20B68D5F89020C5F8983093
:10274000636210231361166916F01006FBD1122084
:10275000FFF776F9D4F8003823F4FE63C4F80038A4
:10276000A36943F4402343F01003A3610923C4F891
:102770001038C4F814380B4BEB604FF0C043C4F86A
:10278000103B094BC4F8003BC4F81069C4F8003989
:10279000D5F8983003F1100243F48013C5F898205F
:1027A000A362F8BD903B000840800010D0F8902054
:1027B00090F88A10D2F8003823F4FE6343EA01133C
:1027C000C2F80038704700002DE9F84300EB8103A0
:1027D000D0F890500C468046DA680FFA81F948012B
:1027E000166806F00306731E022B05EB41134FF02B
:1027F000000194BFB604384EC3F8101B4FF001011E
:1028000004F1100398BF06F1805601FA03F39169B1
:1028100098BF06F5004600293AD0578A04F15801BE
:10282000374349016F50D5F81C180B430021C5F8F8
:102830001C382B180127C3F81019A7405369611ED3
:102840009BB3138A928B9B08012A88BF5343D8F805
:102850009820981842EA034301F140022146C8F843
:102860009800284605EB82025360FFF76FFE08EBE5
:102870008900C3681B8A43EA845348341E436401B9
:102880002E51D5F81C381F43C5F81C78BDE8F883D5
:1028900005EB4917D7F8001B21F40041C7F8001BCE
:1028A000D5F81C1821EA0303C0E704F13F030B4AE3
:1028B0002846214605EB83035A60FFF747FE05EBE8
:1028C0004910D0F8003923F40043C0F80039D5F896
:1028D0001C3823EA0707D7E7008000100004000235
:1028E000D0F894201268C0F89820FFF7C7BD000008
:1028F0005831D0F8903049015B5813F4004004D0AF
:1029000013F4001F0CBF0220012070474831D0F89B
:10291000903049015B5813F4004004D013F4001FB9
:102920000CBF02200120704700EB8101CB68196ABF
:102930000B6813604B6853607047000000EB810325
:1029400030B5DD68AA691368D36019B9402B84BF1C
:10295000402313606B8A1468D0F890201C4402EB6B
:102960004110013C09B2B4FBF3F46343033323F099
:10297000030343EAC44343F0C043C0F8103B2B6851
:1029800003F00303012B0ED1D2F8083802EB4110FB
:1029900013F4807FD0F8003B14BF43F0805343F022
:1029A0000053C0F8003B02EB4112D2F8003B43F069
:1029B0000443C2F8003B30BD2DE9F041D0F89060EF
:1029C00005460C4606EB4113D3F8087B3A07C3F8DB
:1029D000087B08D5D6F814381B0704D500EB810313
:1029E000DB685B689847FA071FD5D6F81438DB0711
:1029F0001BD505EB8403D968CCB98B69488A5A6822
:102A0000B2FBF0F600FB16228AB91868DA68904229
:102A10000DD2121AC3E90024202383F31188214622
:102A20002846FFF78BFF84F31188BDE8F08101236E
:102A300003FA04F26B8923EA02036B81CB68002B53
:102A4000F3D021462846BDE8F041184700EB81034A
:102A50004A0170B5DD68D0F890306C692668E66090
:102A600056BB1A444FF40020C2F810092A6802F03D
:102A70000302012A0AB20ED1D3F8080803EB42146C
:102A800010F4807FD4F8000914BF40F0805040F06B
:102A90000050C4F8000903EB4212D2F8000940F0DC
:102AA0000440C2F800090122D3F8340802FA01F107
:102AB0000143C3F8341870BD19B9402E84BF4020BB
:102AC000206020681A442E8A8419013CB4FBF6F475
:102AD00040EAC44040F00050C6E700002DE9F04154
:102AE000D0F8906004460D4606EB4113D3F8087900
:102AF000C3F80879FB071CD5D6F81038DA0718D5C3
:102B000000EB8103D3F80CC0DCF81430D3F800E0FC
:102B1000DA6896451BD2A2EB0E024FF000081A604D
:102B2000C3F80480202383F31188FFF78FFF88F315
:102B300011883B0618D50123D6F83428AB40134240
:102B400012D029462046BDE8F041FFF7C3BC01235F
:102B500003FA01F2038923EA02030381DCF8083057
:102B6000002BE6D09847E4E7BDE8F0812DE9F84F67
:102B7000D0F8905004466E69AB691E4016F4805838
:102B80006E6103D0BDE8F84FFEF740BC002E12DAAC
:102B9000D5F8003E9F0705D0D5F8003E23F003038B
:102BA000C5F8003ED5F80438204623F00103C5F8E7
:102BB0000438FEF757FC300505D52046FFF75EFCCC
:102BC0002046FEF73FFCB1040CD5D5F8083813F0C9
:102BD000060FEB6823F470530CBF43F4105343F417
:102BE000A053EB60320704D56368DB680BB1204665
:102BF0009847F30200F1BA80B70226D5D4F8909036
:102C000000274FF0010A09EB4712D2F8003B03F40A
:102C10004023B3F5802F11D1D2F8003B002B0DDA01
:102C200062890AFA07F322EA0303638104EB87034C
:102C3000DB68DB6813B13946204698470137D4F882
:102C40009430FFB29B689F42DDD9F00619D5D4F8C5
:102C50009000026AC2F30A1702F00F0302F4F012A6
:102C6000B2F5802F00F0CC80B2F5402F09D104EBF3
:102C70008303002200F58050DB681B6A974240F016
:102C8000B2803003D5F8185835D5E90303D50021B3
:102C90002046FFF791FEAA0303D501212046FFF746
:102CA0008BFE6B0303D502212046FFF785FE2F0321
:102CB00003D503212046FFF77FFEE80203D5042158
:102CC0002046FFF779FEA90203D505212046FFF72C
:102CD00073FE6A0203D506212046FFF76DFE2B0224
:102CE00003D507212046FFF767FEEF0103D5082132
:102CF0002046FFF761FE700340F1A980E90703D584
:102D000000212046FFF7EAFEAA0703D5012120464D
:102D1000FFF7E4FE6B0703D502212046FFF7DEFE36
:102D20002F0703D503212046FFF7D8FEEE0603D573
:102D300004212046FFF7D2FEA80603D50521204630
:102D4000FFF7CCFE690603D506212046FFF7C6FE35
:102D50002A0603D507212046FFF7C0FEEB0576D5EE
:102D600020460821BDE8F84FFFF7B8BED4F8909090
:102D700000274FF0010AD4F894305FFA87FB9B6874
:102D80009B453FF639AF09EB4B13D3F8002902F40A
:102D90004022B2F5802F24D1D3F80029002A20DA6E
:102DA000D3F8002942F09042C3F80029D3F8002953
:102DB000002AFBDB5946D4F89000FFF7C7FB2289B5
:102DC0000AFA0BF322EA0303238104EB8B03DB688B
:102DD0009B6813B159462046984759462046FFF74D
:102DE00079FB0137C7E7910701D1D0F80080072AA6
:102DF00002F101029CBF03F8018B4FEA18283DE75E
:102E000004EB830300F58050DA68D2F818C0DCF8D0
:102E10000820DCE9001CA1EB0C0C00218F4208D13A
:102E2000DB689B699A683A449A605A683A445A60E7
:102E300027E711F0030F01D1D0F800808C4501F194
:102E4000010184BF02F8018B4FEA1828E6E7BDE8CC
:102E5000F88F000008B50348FFF788FEBDE808407A
:102E6000FFF784BAAC40002008B50348FFF77EFEA8
:102E7000BDE80840FFF77ABA48410020D0F890300A
:102E800003EB4111D1F8003B43F40013C1F8003BC0
:102E900070470000D0F8903003EB4111D1F80039B1
:102EA00043F40013C1F8003970470000D0F89030A7
:102EB00003EB4111D1F8003B23F40013C1F8003BB0
:102EC00070470000D0F8903003EB4111D1F8003981
:102ED00023F40013C1F8003970470000090100F124
:102EE0006043012203F56143C9B283F8001300F087
:102EF0001F039A4043099B0003F1604303F56143BC
:102F0000C3F880211A60704730B50433039C017206
:102F1000002104FB0325C160C0E90653049B036341
:102F2000059BC0E90000C0E90422C0E90842C0E9ED
:102F30000A11436330BD00000022416AC260C0E94B
:102F40000411C0E90A226FF00101FEF7E9BD00009B
:102F5000D0E90432934201D1C2680AB9181D704702
:102F600000207047036919600021C2680132C26005
:102F7000C269134482699342036124BF436A0361B7
:102F8000FEF7C2BD38B504460D46E3683BB1626941
:102F90000020131D1268A3621344E36207E0237A42
:102FA00033B929462046FEF79FFD0028EDDA38BDEB
:102FB0006FF00100FBE70000C368C269013BC3601A
:102FC0004369134482699342436124BF436A436166
:102FD00000238362036B03B11847704770B5202349
:102FE000044683F31188866A3EB9FFF7CBFF054696
:102FF00018B186F31188284670BDA36AE26A13F8F7
:10300000015B9342A36202D32046FFF7D5FF002362
:1030100083F31188EFE700002DE9F84F04460E46D0
:10302000174698464FF0200989F311880025AA46D3
:10303000D4F828B0BBF1000F09D141462046FFF774
:10304000A1FF20B18BF311882846BDE8F88FD4E9A1
:103050000A12A7EB050B521A934528BF9346BBF102
:10306000400F1BD9334601F1400251F8040B914245
:1030700043F8040BF9D1A36A403640354033A362CC
:10308000D4E90A239A4202D32046FFF795FF8AF338
:103090001188BD42D8D289F31188C9E730465A4613
:1030A000FDF79CFEA36A5E445D445B44A362E7E7D0
:1030B00010B5029C0433017204FB0321C460C0E913
:1030C00006130023C0E90A33039B0363049BC0E992
:1030D0000000C0E90422C0E90842436310BD0000BB
:1030E000026A6FF00101C260426AC0E90422002254
:1030F000C0E90A22FEF714BDD0E904239A4201D1A7
:10310000C26822B9184650F8043B0B607047002093
:1031100070470000C3680021C2690133C36043697E
:10312000134482699342436124BF436A4361FEF7BB
:10313000EBBC000038B504460D46E3683BB123699B
:1031400000201A1DA262E2691344E36207E0237AB9
:1031500033B929462046FEF7C7FC0028EDDA38BD12
:103160006FF00100FBE7000003691960C268013AD3
:10317000C260C269134482699342036124BF436AF7
:10318000036100238362036B03B11847704700009B
:1031900070B520230D460446114683F31188866AD4
:1031A0002EB9FFF7C7FF10B186F3118870BDA36A6F
:1031B0001D70A36AE26A01339342A36204D3E169FA
:1031C00020460439FFF7D0FF002080F31188EDE797
:1031D0002DE9F84F04460D46904699464FF0200AD7
:1031E0008AF311880026B346A76A4FB9494620469C
:1031F000FFF7A0FF20B187F311883046BDE8F88FB4
:10320000D4E90A073A1AA8EB0607974228BF1746DF
:10321000402F1BD905F1400355F8042B9D4240F87F
:10322000042BF9D1A36A40364033A362D4E90A23C0
:103230009A4204D3E16920460439FFF795FF8BF3E6
:1032400011884645D9D28AF31188CDE729463A46F6
:10325000FDF7C4FDA36A3D443E443B44A362E5E759
:10326000D0E904239A4217D1C3689BB1836A8BB11A
:10327000043B9B1A0ED01360C368013BC360C36953
:103280001A4483699A42026124BF436A036100239E
:1032900083620123184670470023FBE700F0DAB889
:1032A000034B002258631A610222DA60704700BFA4
:1032B000000C0040014B0022DA607047000C004017
:1032C000014B5863704700BF000C0040014B586A27
:1032D000704700BF000C00404B6843608B68836000
:1032E000CB68C3600B6943614B6903628B694362BE
:1032F0000B6803607047000008B53C4B40F2FF715B
:103300003B48D3F888200A43C3F88820D3F88820A4
:1033100022F4FF6222F00702C3F88820D3F8882045
:10332000D3F8E0200A43C3F8E020D3F808210A4389
:10333000C3F808212F4AD3F808311146FFF7CCFF14
:1033400000F5806002F11C01FFF7C6FF00F5806008
:1033500002F13801FFF7C0FF00F5806002F154016F
:10336000FFF7BAFF00F5806002F17001FFF7B4FFCC
:1033700000F5806002F18C01FFF7AEFF00F5806080
:1033800002F1A801FFF7A8FF00F5806002F1C40177
:10339000FFF7A2FF00F5806002F1E001FFF79CFF5C
:1033A00000F5806002F1FC01FFF796FF02F58C71D9
:1033B00000F58060FFF790FF00F000F90E4BD3F8A6
:1033C000902242F00102C3F89022D3F8942242F0F6
:1033D0000102C3F894220522C3F898204FF06052EE
:1033E000C3F89C20054AC3F8A02008BD0044025839
:1033F00000000258CC3B000800ED00E01F0008036D
:1034000008B500F0C9FAFEF7DFFA0F4BD3F8DC205D
:1034100042F04002C3F8DC20D3F8042122F040023D
:10342000C3F80421D3F80431084B1A6842F00802AB
:103430001A601A6842F004021A60FEF749FFBDE8FC
:103440000840FEF7E9BC00BF0044025800180248DB
:1034500070470000114BD3F8E82042F00802C3F88F
:10346000E820D3F8102142F00802C3F810210C4ADA
:10347000D3F81031D36B43F00803D363C722094B51
:103480009A624FF0FF32DA6200229A615A63DA6080
:103490005A6001225A611A60704700BF0044025806
:1034A0000010005C000C0040094A08B51169D3689F
:1034B0000B40D9B29B076FEA0101116107D52023A8
:1034C00083F31188FEF7A0FA002383F3118808BD67
:1034D000000C0040384B4FF0FF31D3F88020C3F888
:1034E0008010D3F880200022C3F88020D3F8800019
:1034F000D3F88400C3F88410D3F88400C3F8842080
:10350000D3F88400D86F40F0FF4040F4FF0040F44F
:103510003F5040F03F00D867D86F20F0FF4020F4C4
:10352000FF0020F43F5020F03F00D867D86FD3F859
:1035300088006FEA40506FEA5050C3F88800D3F813
:103540008800C0F30A00C3F88800D3F88800D3F8D5
:103550009000C3F89010D3F89000C3F89020D3F8EF
:103560009000D3F89400C3F89410D3F89400C3F8F3
:103570009420D3F89400D3F89800C3F89810D3F8A7
:103580009800C3F89820D3F89800D3F88C00C3F8BB
:103590008C10D3F88C00C3F88C20D3F88C00D3F8AF
:1035A0009C00C3F89C10D3F89C10C3F89C20D3F85F
:1035B0009C3000F0C9B900BF00440258614B0122A1
:1035C000C3F80821604BD3F8F42042F00202C3F89C
:1035D000F420D3F81C2142F00202C3F81C2102227D
:1035E000D3F81C31594BDA605A689104FCD5584A1B
:1035F0001A6001229A60574ADA6000221A614FF479
:1036000040429A61514B9A699204FCD51A6842F47F
:1036100080721A604C4B1A6F12F4407F04D04FF442
:1036200080321A6700221A671A6842F001021A6093
:10363000454B1A685007FCD500221A611A6912F02E
:103640003802FBD1012119604FF0804159605A675F
:10365000414ADA62414A1A611A6842F480321A60B9
:10366000394B1A689103FCD51A6842F480521A60EB
:103670001A689204FCD53A4A3A499A6200225A637F
:1036800019633949DA6399635A64384A1A64384AC3
:10369000DA621A6842F0A8521A602B4B1A6802F0DC
:1036A0002852B2F1285FF9D148229A614FF488621A
:1036B000DA6140221A622F4ADA644FF080521A65AA
:1036C0002D4A5A652D4A9A6532232D4A1360136894
:1036D00003F00F03022BFAD11B4B1A6942F00302CD
:1036E0001A611A6902F03802182AFAD1D3F8DC20DC
:1036F00042F00052C3F8DC20D3F8042142F000521B
:10370000C3F80421D3F80421D3F8DC2042F080422E
:10371000C3F8DC20D3F8042142F08042C3F804212E
:10372000D3F80421D3F8DC2042F00042C3F8DC20B7
:10373000D3F8042142F00042C3F80421D3F8043145
:10374000704700BF008000510044025800480258F2
:1037500000C000F0020000010000FF010088900896
:1037600012102000630209012C020400470405081E
:10377000FD0BFF01200000200010E000000101000F
:10378000002000524FF0B04208B5D2F8883003F064
:103790000103C2F8883023B1044A13680BB15068A2
:1037A0009847BDE80840FEF7E1BD00BFFC4100209E
:1037B0004FF0B04208B5D2F8883003F00203C2F8E7
:1037C000883023B1044A93680BB1D0689847BDE8AC
:1037D0000840FEF7CBBD00BFFC4100204FF0B042D7
:1037E00008B5D2F8883003F00403C2F8883023B15A
:1037F000044A13690BB150699847BDE80840FEF7C9
:10380000B5BD00BFFC4100204FF0B04208B5D2F872
:10381000883003F00803C2F8883023B1044A936962
:103820000BB1D0699847BDE80840FEF79FBD00BFC7
:10383000FC4100204FF0B04208B5D2F8883003F0C8
:103840001003C2F8883023B1044A136A0BB1506ADE
:103850009847BDE80840FEF789BD00BFFC41002045
:103860004FF0B04310B5D3F8884004F47872C3F831
:103870008820A30604D5124A936A0BB1D06A9847F0
:10388000600604D50E4A136B0BB1506B98472106A6
:1038900004D50B4A936B0BB1D06B9847E20504D566
:1038A000074A136C0BB1506C9847A30504D5044A22
:1038B000936C0BB1D06C9847BDE81040FEF756BD35
:1038C000FC4100204FF0B04310B5D3F8884004F419
:1038D0007C42C3F88820620504D5164A136D0BB1EB
:1038E000506D9847230504D5124A936D0BB1D06DE6
:1038F0009847E00404D50F4A136E0BB1506E9847F9
:10390000A10404D50B4A936E0BB1D06E98476204A4
:1039100004D5084A136F0BB1506F9847230404D5A0
:10392000044A936F0BB1D06F9847BDE81040FEF783
:103930001DBD00BFFC41002008B5FFF7B5FDBDE887
:103940000840FEF713BD0000062108B50846FFF742
:10395000C5FA06210720FFF7C1FA06210820FFF764
:10396000BDFA06210920FFF7B9FA06210A20FFF760
:10397000B5FA06211720FFF7B1FA06212820FFF734
:10398000ADFA09217A20FFF7A9FA07213220BDE814
:103990000840FFF7A3BA000008B5FFF79BFD00F051
:1039A0000BF8FDF7C1FCFDF793FBFFF751FDBDE8F8
:1039B0000840FFF773BC00000023054A1946013395
:1039C000102BC2E9001102F10802F8D1704700BFC4
:1039D000FC41002010B501390244904201D1002081
:1039E00005E0037811F8014FA34201D0181B10BD68
:1039F0000130F2E7034611F8012B03F8012B002AEE
:103A0000F9D1704753544D333248373F3F3F00534D
:103A1000544D3332483734332F37353300000000EC
:103A2000000000004D100008391000087510000853
:103A3000611000086D1000085910000845100008BA
:103A40003110000881100008000000000100000093
:103A5000000000006D61696E0000000069646C6523
:103A6000000000005C3A0008F823002070250020C8
:103A700001000000C51900080000000041726475D3
:103A800050696C6F740025424F415244252D424CC1
:103A9000002553455249414C25000000020000001A
:103AA000000000006D120008DD1200084000400018
:103AB000183E0020283E0020020000000000000008
:103AC00003000000000000002513000800000000B3
:103AD00010000000383E002000000000010000003F
:103AE00000000000AC40002001010200B51D0008EC
:103AF000C51C0008611D0008451D000843000000AA
:103B0000043B000809024300020100C0320904001E
:103B1000000102020100052400100105240100013A
:103B2000042402020524060001070582030800FFA1
:103B300009040100020A000000070501024000001C
:103B4000070581024000000012000000503B000801
:103B50001201100102000040091241570002010247
:103B6000030100000403090425424F41524425008B
:103B70004B616B75746548374D696E690030313241
:103B80003334353637383941424344454600000026
:103B9000000000007914000831170008DD17000844
:103BA00040004000E4410020E4410020010000000A
:103BB000F4410020800000004001000008000000E7
:103BC0000001000000040000080000000001802A3D
:103BD00000000000AAAAAAAA00010024FFFF00001A
:103BE0000000000000A00A000000400100000000EA
:103BF000AAAAAAAA00000001FFFF0000000000001E
:103C0000000000001000000400000000AAAAAAAAF8
:103C100000000008FBDF00000000000000000000C2
:103C20000000000000000000AAAAAAAA00000000EC
:103C3000FFFF000000000000000000000001000085
:103C400000000000AAAAAAAA00010000FFFF0000CD
:103C50000000000000000000000000000000000064
:103C6000AAAAAAAA00000000FFFF000000000000AE
:103C7000000000000000000000000000AAAAAAAA9C
:103C800000000000FFFF0000000000000000000036
:103C90000000000000000000AAAAAAAA000000007C
:103CA000FFFF000000000000000000000000000016
:103CB00000000000AAAAAAAA00000000FFFF00005E
:103CC00000000000000000000000000000000000F4
:103CD000AAAAAAAA00000000FFFF0000000000003E
:103CE000000000000000000000000000AAAAAAAA2C
:103CF00000000000FFFF00000000000000000000C6
:103D0000220400000000000000001A000000000073
:103D1000FF00000000000000043A00083F0000001F
:103D2000500400000F3A00083F0000000096000019
:103D300000000800960000000008000004000000D9
:103D4000643B0008000000000000000000000000CC
:0C3D500000000000000000000000000067
:00000001FF
